:1000000034C041C040C03FC03EC03DC03CC03BC00A
:100010003AC039C049C135C125C11BC116C112C181
:100020001FC11BC118C14AC17C919EA6B0FFA1A3EC
:10003000A3A3A3A1A1A1A1A1A1A1A1A1A1A1A1A1AA
:10004000A1A1031496FFFF000000000000000000C3
:1000500000060A0B0600000003216EFFFDFCFBFEFC
:10006000F7FAF9F8F6F5FEF9FBFF11241FBECFE908
:10007000CDBF10E0A0E6B0E001C01D92A236B107EE
:10008000E1F770D098C1BCCF26EB33E003C0F90193
:100090003197F1F70197D8F70895009709F0F4CF59
:1000A00080E991E00197F1F7089588EE93E0ECCFB5
:1000B000CF93C09161008C2F8F5F8F73809361000D
:1000C0006091600090E069D16FEF8C2F90E0CF914C
:1000D00064C1811104C0611102C091EA9FBD89BD54
:1000E00066BF0895FC01E25DFF4FE491EFBDFC01A6
:1000F000EE5BFF4F6491FC01EA5AFF4F8491E9CF18
:10010000369A3699FECF85B10895CF93DF931F922B
:10011000CDB7DD279FEF99BD16BE90E06983BDDFA7
:1001200081EA8FBD19BC16BE6981862F90E00F90C1
:10013000DF91CF91B2CFCF93DF93D82FC4E060E0AF
:100140008D2FC7DF85E090E09FDF6D2F80E0C1DF5E
:1001500081E490E099DFC15091F780ED92E0DF916A
:10016000CF9192CFA39A83E687B986EC86B9369968
:10017000FECF369A3699FECFD5B180E188BBB99AC9
:10018000B89A81EA8FBD81E083BF1092610009C0F7
:100190008C2F90E0FAD08F3F09F0F4C0CF5FC0936E
:1001A0006100C0916100C03498F3DB3F88F0E091BA
:1001B0006000EF5FE0936000E63009F41CC0E031BE
:1001C000E0F0F0E0EF5BFF4FE491E093600015C0DA
:1001D000DF3B88F080916000803109F40CC08630EC
:1001E00011F48FE005C0882311F0815001C083E134
:1001F0008093600002C0109260005ADFBB9AC39ADD
:10020000A29A81E687B986EC86B9369AD0E010E0EA
:1002100001EA84E1F82E93E6E92E21E4D22E8091C2
:100220006000E82FF0E0EA5AFF4FC4914C2F50E0F5
:10023000FA01E55FF109EA30F10508F05EC0E65F1A
:10024000FF4F09946FE481E002C069E280E05DDF66
:100250006DC06FE0FBCF84E001C089E16CDF66C058
:100260008FEFFCCF69EF81E050DF69EF81E04DDF78
:100270005AC0813218F06D2D6C1B01C0682FC82F39
:1002800002C0C0E060E0655E660F81E03EDF8C2F5B
:100290008F5F823471F74AC0823318F06E2D6C1B69
:1002A00001C0682FC82F02C0C0E060E0675F80E037
:1002B0002CDF8C2F8F5F843679F738C00FBD19BCC7
:1002C00016BEF3DE1DDFC0E001C0CF5FEC2FF0E013
:1002D000E85DFF4FE491E817C0F30CC019BCF6BE0F
:1002E00084E690E0D1DE0FBD19BC16BE80E991E036
:1002F000CBDEC150C111F2CF19C090E0F3DE1F5F19
:100300001F3188F0C43678F080916000863010F09C
:1003100084E001C08150809360008091600090E093
:10032000E1DEC6DE10E084EF91E0AEDE349B77CFF5
:1003300085B1843720F5DF5FD83010F1C0916000BF
:10034000C63098F4CC2311F0C15010C00FBD19BCB9
:1003500016BE85B7877E806185BF85B7806285BF01
:10036000889585B78F7D85BF01C0C2E08C2F90E056
:10037000B9DEC09360009CDE8AEF90E085DED0E0BD
:10038000369A4DCF8093600010CFE199FECF1FBA0F
:100390008EBBE09A99278DB30895262FE199FECF61
:1003A0001CBA1FBA8EBB2DBB0FB6F894E29AE19A25
:0A03B0000FBE01960895F894FFCFE8
:00000001FF
